S018000064656D6F70726F675F786D63313430302E7372656343
S31510003000500500201D30001000000000A5300010F3
S315100030100018040000010000EE11AA55124885465A
S315100030201249134A134B00F018F8134880471349F6
S31510003030134A144B00F011F81349144A144B00F0BC
S315100030400CF81449144A0020521A02DD043A88502A
S31510003050FCDC12488047124880479B1A03DD043B6C
S31510003060C858D050FBDC704750050020783C001043
S315100030700C0000205001002081310010BC3D0010D2
S315100030805005002050050020BC3D001050050020C2
S315100030905005002050050020D40500202D3C0010BE
S315100030A0A53B0010FEE70000024A936E01218B43F8
S315100030B0936670470000014000487047002D3101AB
S315100030C038B51D4B1B681B041B0E1C4A136026D0FB
S315100030D019480268FF211140194C2160C269032565
S315100030E02A40120211432160C269920508D49B023C
S315100030F0C918144800F07AFA0001134B18601AE048
S31510003100FFF7DAFF80010D4B196889020C4B1B681B
S31510003110C91800F06BFA00010B4B18600BE0064B58
S31510003120DB699B0503D4094A074B1A6003E0FFF7D6
S31510003130C3FF054B186038BD000301405005002041
S315100031405405002000001BB7FC3F0020006CDC0279
S3151000315008B50749C0234B62064BD869064A024098
S31510003160DA61064A1A60C3234B62FFF7A9FF08BD4E
S315100031700000014000030140FFFDFFFF0001F13F89
S3151000318008B5FFF791FFFFF7E3FF08BDF0B54F460F
S315100031904646C0B48B08994604339B001E58032537
S315100031A00D40ED00FC27AF40BE431E50436F4F004D
S315100031B00326BE40B3434367CB0810339B001C580D
S315100031C007260E40B6000427B740BC431C501F58B4
S315100031D0BC465778B7403E1C67463E431E500C4BC4
S315100031E0984204D1036E01268E40B343036653689A
S315100031F08B4043604B4604339B0019581278AA4003
S31510003200151C0D431D500CBC90469946F0BDC0468A
S3151000321000020440C322014B5A627047000001406D
S31510003220C022034B5A62024B5B6A5B07FBD47047A2
S315100032300000014010B5041CFFF7F2FF054B1A6998
S3151000324014431C61034B1B685B00FBD4FFF7E2FFC2
S3151000325010BDC04600030140014B18687047C046B8
S31510003260FC3F0020F0B55F465646C0B485B0834695
S315100032700F1C454B9A4600230293039301253AE00F
S315100032803B689800C0184000291C00F0AFF9019067
S315100032907C68211C00F0AAF9061C0A2100F0B0F97E
S315100032A0052905D9301C0A2100F0A0F9461C04E0B6
S315100032B0301C0A2100F09AF9061C002E06D0B10027
S315100032C089194900019800F091F904E001980A2142
S315100032D000F08CF90126A04201D3041B00E0241A49
S315100032E0142E07D8A24505D9284B9C4206D9A246CA
S315100032F0029603950135402DC2D901E00296039539
S31510003300214E0124402512E0681C1F4B5843029998
S3151000331000F06CF93B89834201D8C21A00E01A1AF0
S31510003320964201D9161C2C1C984202D3013D022D3F
S31510003330EAD8029B191B5B461B684022134358466A
S3151000334003608B1E1903E023DB011940081C7B89DF
S31510003350013B9B01FF210B401843071C013C240233
S31510003360F0231B011C402743039B013BC0390B4034
S315100033701F435B461F611B6893435A46136005B093
S315100033800CBC92469B46F0BD10270000E7030000D8
S3151000339010B5E2235B00C4583D33FF331C42F8D10D
S315100033A00131120402231A4309061143C333FF33B2
S315100033B0C15010BD10B5041C80208003FFF73AFFE2
S315100033C0236801229343236023689B07FCD410BD16
S315100033D010B5E422520083580F24A3431943815099
S315100033E010BDC046E4235B00C058BA3BFF3B1840F3
S315100033F07047C04608B5FFF7F5FF012802D002282E
S3151000340003D005E0FFF728FF03E0FFF755FE00E0C5
S31510003410002008BDF0B5474680B4051C0C1C161CD0
S31510003420FFF7C8FF281C211CFFF7D2FF281CFFF747
S31510003430E1FF041C311C00F0D9F88027FF003F1A69
S31510003440194B9F4200D91F1C8021C900C91B201C83
S3151000345000F0CCF88046B009A4098002211C00F0C7
S31510003460C5F8114B984200D9181C4443A40AA4016C
S315100034704346F21A341B002394425B41DBB2002B05
S3151000348000D0381C002B01D0012300E00223E9688C
S31510003490064A0A40EA60EA689B0318431043E8604C
S315100034A004BC9046F0BDC046FF030000003CFFFF81
S315100034B010B5037E012B18D103682022DA61046847
S315100034C021680B4B1940037B1B06F0221205134093
S315100034D00B432360036802691A61036842695A61E3
S315100034E00368044ADA61002000E0032010BDC046DC
S315100034F0FFFFFFF04000280010B50268204BD318DC
S31510003500990A49039B05DB0E1B020B4394681D4960
S3151000351021409160026891680B439360037E012BF2
S315100035202CD803682022DA61C3799B060ED4416831
S315100035304B0F5A078B0413430268936181684B0F34
S315100035405A078B0413430268D36005E00368426888
S315100035509A6103688268DA60041C037E012B06D127
S31510003560FFF7A6FF236880221205DA6103E00368DD
S3151000357080221201DA612368034ADA6110BDC0465F
S3151000358000F0FBAFFF00FFFF4000A0060268D16904
S31510003590D3695B07DB0F09050FD4012B0FD0136915
S315100035A0036153694361D169D3691B07DB0F49076F
S315100035B007D5002BF3D1002004E0032002E00220FF
S315100035C000E000207047C04630B58B0804339B00DE
S315100035D01C5803252940C900F9358D40AC431C50B1
S315100035E01C588A40111C2143195030BD034B04222C
S315100035F05A6318625962986A7047C04600000340C1
S31510003600034B04225A6318625962D96A986A704742
S315100036100000034070B5051C0E1C00F0DBF8F479B1
S31510003620002C00D11034281C3168221C00F03CF804
S31510003630B379013B5B006408013424021C43114B2F
S315100036401C43EC633379013B1B0681225200134362
S315100036506B637379002B05D06A6B013B1B04134314
S315100036606B6305E0696B3279531E1B040B436B6366
S31510003670A023DB00AB6301235B42EB6433892B642D
S3151000368070BDC0460100030086235B00C258E023CC
S31510003690DB041A4202D1406D80B203E08E235B0038
S315100036A0C05880B27047C046F0B55F464E46C0B4AB
S315100036B083B063293DD9002A3DD0151C0C1C8346C6
S315100036C0FFF7CAFD6421FFF791FF8146201C642194
S315100036D0FFF78CFF071C1B4E012301930093341C2C
S315100036E011E048466043291C7943FFF77FFF830AA0
S315100036F08005800D134A934204D8B04202D2061CAC
S3151000370001930094013C002CEBD180231B02009FF7
S315100037101F435B461F615A690B4B1340013DAD02B7
S315100037201D43019E013E360435435B465D61002014
S3151000373002E0012000E0012003B00CBC91469B463C
S31510003740F0BDC046FF030000EF8000FC70B5842575
S315100037506D004659064C344044514659054C264096
S315100037601B02194314060A1C22433243425170BDF0
S31510003770FFFFFFF8C0C0FFF870B586256D004659EB
S31510003780084C344044514659074C26401B021943F5
S3151000379014060A1C22433243802149050A4342512A
S315100037A070BDC046FFFFFFF8C0C0FFEF08B5074B5E
S315100037B0984203D10820FFF73DFD06E0044B9842DE
S315100037C003D18020C002FFF735FD08BD0800004870
S315100037D00840004810B5041C9023DB05984202D01F
S315100037E00C4B984203D10C48FFF7E0FF08E00B4B57
S315100037F0984202D00A4B984202D10A48FFF7D6FFE8
S315100038000323E360E368DB07FCD5236C0F229343A5
S31510003810236410BD0002004808000048004000481C
S3151000382000420048084000487047C04630B589B08D
S3151000383001A9E1231B02019308230B714B71073B6E
S315100038408B710F33CB7100230B81174C201CFFF7A4
S31510003850E1FE06AA00231370144D281C0321FFF75E
S3151000386095FC04AA9C231370281C0221FFF78EFCDA
S31510003870E36950229343E361E369493A9343E36171
S31510003880201C1021033A0123FFF760FF201C0021A2
S3151000389004220123FFF770FF236C0F2293430D3A86
S315100038A01343236409B030BD0002004800010440F0
S315100038B070B588B0FFF7D0FC041C00E064003E4BE6
S315100038C09C42FBD900E064083C4B9C42FBD83C4828
S315100038D00121221CFFF79EFD01A90194394B4B6073
S315100038E0FA235B010B8101254D81374C201CFFF714
S315100038F0B9FC226840231343236023681D432560C7
S31510003900324A33481060D3793F210B40BF390B43FD
S31510003910D37153685B0F5B072E4C2343536091683A
S31510003920490F4907214391601B0E2024A343D371ED
S31510003930090E20231943D172C368802189050B43D0
S31510003940C36008231373002305E0204AD218002110
S3151000395011740133DBB2072BF7D91C480026067603
S31510003960FFF7CAFD164801210122FFF711FD164C7B
S3151000397023684025AB4323602368012293432360C9
S3151000398006AA1670144E301C0821FFF7FFFB04AA76
S31510003990A4231370301C0921FFF7F8FB23682B436F
S315100039A02360E36807229343053A1343E3602368D1
S315100039B0AB43236008B070BDFF1AB700000E27078F
S315100039C00000045020A1070000030450A8050020A1
S315100039D020100450670600000004044010B58A2326
S315100039E05B00064AD3581B0706D4041C101CFFF7AD
S315100039F04BFE2070012000E0002010BD00020048A0
S31510003A0008B5FFF713FFFFF753FF08BDBFF34F8F3E
S31510003A10034A044BDA60BFF34F8FC046FDE7C0463A
S31510003A200400FA0500ED00E008B5214B1B78002BC9
S31510003A3013D12048FFF7D2FF012837D11D4B1B7831
S31510003A40002B33D000F0E4F81B4B18600122184B02
S31510003A501A700022194B1A7028E0184B187801308A
S31510003A60144B1818FFF7BAFF012815D1134A13780B
S31510003A700133DBB213700F4A1278934216D100222B
S31510003A800B4B1A700B4B5B78FF2B0FD1094B9B78A6
S31510003A90002B0BD1FFF7BAFF00F0BAF8064B1B68E4
S31510003AA06433984202D90022014B1A7008BDC046F1
S31510003AB09D05002058050020A00500209C0500202B
S31510003AC000B583B0174B1B68DB69DB071AD51548A1
S31510003AD0FFF75CFD00280AD000220EE0114AD2182A
S31510003AE0127C6946CA540133DBB2012201E000227E
S31510003AF000230C49097B9942F0D80A4B1B68012117
S31510003B00D96100E00022012A09D16B461B78FF2BF0
S31510003B1005D16B465B78002B01D1FFF777FF03B019
S31510003B2000BDC046A805002008B5FFF77DFFFFF7CA
S31510003B30C7FF08BD10B5044C201C00218022FFF7DA
S31510003B4043FD0123636010BD0004044008B500F076
S31510003B505FF80E4B1B68C31AF422FF32934214D936
S31510003B600B4B1B78002B08D1F33AFF3A084B1A700F
S31510003B7080225202074B5A6005E00022044B1A704D
S31510003B800132044B5A60014B186008BDC80500206D
S31510003B90CC0500200004044008B5FFF7CBFF00F069
S31510003BA011F808BD08B5FFF7F7FFFFF729FFFFF774
S31510003BB0CDFFFFF7B9FFFAE7014B18607047C04613
S31510003BC0D005002008B50E4B1868FA218900FFF7BA
S31510003BD00DFD01380B4B98420DD80B4A50600B491E
S31510003BE00B6A1B021B0AC020000603430B6200234C
S31510003BF09360073313600020FFF7DEFF08BDC04651
S31510003C00FC3F0020FFFFFF0010E000E000ED00E0A9
S31510003C10014B18687047C046D0050020024A136849
S31510003C20013313607047C046D00500200E4B70B5A7
S31510003C3000251E1C0D4CE41AA410A54204D0AB009E
S31510003C40F35898470135F8E7FFF7EEFD084B0025C6
S31510003C501E1C084CE41AA410A54204D0AB00F3585D
S31510003C6098470135F8E770BD500500205005002033
S30D10003C7050050020500500204C
S31510003C782C4800470000000000000000000000006B
S31510003C880000000000000000000000000000000016
S31510003C9825480047000000000000000023480047A0
S31510003CA8234800472348004723480047234800472E
S31510003CB8234800472348004723480047234800471E
S31510003CC8234800472348004723480047234800470E
S31510003CD823480047234800472348004723480047FE
S31510003CE823480047234800472348004723480047EE
S31510003CF823480047234800472348004723480047DE
S31510003D0823480047234800472348004723480047CD
S31510003D1823480047234800472348004723480047BD
S31510003D2823480047A5300010A5300010A530001014
S31510003D381D3C0010A5300010A5300010A53000104D
S31510003D48A5300010A5300010A5300010A5300010C1
S31510003D58A5300010A5300010A5300010A5300010B1
S31510003D68A5300010A5300010A5300010A5300010A1
S31510003D78A5300010A5300010A5300010A530001091
S31510003D88A5300010A5300010A5300010A530001081
S31510003D98A5300010A5300010A5300010A530001071
S31510003DA8A5300010A5300010A5300010A530001061
S30910003DB8A53000100C
S7051000301D9D
